:1000000012C02DC02BC02AC029C028C027C026C0BE
:1000100025C024C023C022C021C020C01FC01EC0D4
:100020001DC01CC01BC011241FBECFE5D4E0DEBF25
:10003000CDBF10E0A0E6B0E0E4E4FCE002C0059033
:100040000D92A837B107D9F710E0A8E7B0E001C0DA
:100050001D92AB39B107E1F70CD2F2C5D1CF1F9297
:100060000F920FB60F9211242F933F938F939F936C
:1000700020916000C59A80917B00882349F080918F
:100080007C0082FD206C80917C008F5F80937C00DF
:1000900027FF02C0A89A01C0A8988299FECF12BE7D
:1000A00081E088BF90E431E003C008B600FC15C0D1
:1000B0009999FBCF892F822311F0A89A01C0A898A3
:1000C00012BE38BF829909C0969521F0F1CF08B6CB
:1000D00000FC03C09999FBCFA89881E080937A0037
:1000E000C5989F918F913F912F910F900FBE0F90C8
:1000F0001F901895482F90E820E030E0FB01E20FB8
:10010000F31F892F8423808396952F5F3F4F2830DC
:100110003105A1F70895992787FD9095A92FB92F4B
:10012000BC01CD0120EC3DE540E050E020D52FEFB3
:100130003FE740E050E03AD5822F0895892B71F0D7
:100140002091600080E890E002C0959587956A95BF
:10015000E2F78095822380936000089520916000EB
:1001600080E890E002C0959587956A95E2F7282B84
:10017000209360000895EF92FF920F931F93CF9307
:10018000DF937A01082F10E0C22FD0E080E890E0E2
:100190008C1B9D0B081719071CF481E090E0CEDF43
:1001A000C058DF4FC017D10724F481E090E0B701B9
:1001B000C5DFDF91CF911F910F91FF90EF900895D0
:1001C0009F92AF92BF92CF92DF92EF92FF920F93E6
:1001D0001F93CF93DF935A0169019E2CE82EFF24D1
:1001E00010E0C0E8D0E0CE01801B910BE816F906C4
:1001F00064F481E090E0A2DFC919D109EC16FD0694
:1002000024F481E090E0B60199DF00581F4F0E15ED
:100210001F057CF481E090E0B50190DF892D90E02E
:1002200080589F4F8E159F0524F481E090E0B60121
:1002300085DFDF91CF911F910F91FF90EF90DF90BD
:10024000CF90BF90AF909F900895EF920F938091C1
:100250007800909179008130910509F457C082307F
:10026000910509F4A4C0892B09F0F6C0809199008A
:1002700090E08071907060E070E060DF80919900A4
:1002800090E08870907061E070E058DF8091990094
:1002900090E08078907062E070E050DF809199008B
:1002A00090E08170907063E070E048DF80919A0088
:1002B00090E08170907064E070E040DF80919A007F
:1002C00090E08270907065E070E038DF80919A0075
:1002D00090E08870907066E070E030DF80919A0066
:1002E00090E08470907067E070E028DF8091930068
:1002F00066E070E047E050E028E33DDF8091940045
:1003000064E070E045E050E028E34FC08091990040
:1003100090E08071907060E070E010DF8091990053
:1003200090E08870907061E070E008DF8091990043
:1003300090E08078907062E070E000DF809199003A
:1003400090E08170907063E070E0F8DE80919A0038
:1003500090E08170907064E070E0F0DE80919A002F
:1003600090E08270907065E070E0E8DE80919A0025
:1003700090E08870907066E070E0E0DE80919A0016
:1003800090E08470907067E070E0D8DE8091930018
:1003900066E070E047E050E020E2EDDE80919400FE
:1003A00064E070E045E050E020E2E5DE55C0809179
:1003B000990090E08071907060E070E0BFDE809105
:1003C000990090E08870907061E070E0B7DE8091F5
:1003D000990090E08078907062E070E0AFDE8091EC
:1003E000990090E08170907063E070E0A7DE8091EA
:1003F0009A0090E08170907064E070E09FDE8091E0
:100400009A0090E08270907065E070E097DE8091D5
:100410009A0090E08870907066E070E08FDE8091C6
:100420009A0090E08470907067E070E087DE8091C1
:10043000930066E070E047E050E021E030E000E249
:1004400090E4E92EBDDE8091940064E070E045E028
:1004500050E021E030E0B4DE8091990085FF04C0D7
:1004600081E080937B0002C010927B000F91EF909F
:10047000089578D0FC01909392008093910011BA76
:100480009FEF92BB17BA98BB80E287BBC59881E00B
:1004900084BB95BB85B7836085BF8BB780648BBFFA
:1004A0008BB78F778BBF82E083BF0284F385E02D0B
:1004B000099588E893E120E931E0F9013197F1F7F6
:1004C0000197D9F7E0919100F09192000484F585AD
:1004D000E02D0995E0919100F09192000088F1895A
:1004E000E02D83E990E0099580919900282F84FF01
:1004F00006C082E090E0909379008093780023FF1B
:1005000006C081E090E09093790080937800DFD27C
:10051000789480917A00882321F010927A00E5D2B5
:10052000C59812D38823A9F3E0919100F09192002D
:100530000484F585E02D0995E0919100F0919200F9
:100540000684F785E02D0995882319F3E091910041
:10055000F09192000088F189E02D83E990E00995FF
:1005600074DED7CF81E690E00895009741F0DC017A
:10057000EDE7F0E088E001900D928150E1F7A5E809
:10058000B0E0EDE7F0E088E001900D928150E1F7F6
:1005900008958091750090917600892B31F010922A
:1005A00076001092750081E008958DE790E065E88F
:1005B00070E048E050E037D308950F931F93DF9326
:1005C000CF93CDB7DEB7C850D1400FB6F894DEBF99
:1005D0000FBECDBF80E0E3D1FE01399680E0EF93FE
:1005E000FF9300E810E41023A9F00000A59A000092
:1005F00000000000000000000000000000000000FB
:100600000000A59838E03A95F1F700000000069543
:1006100061F0E8CFA59A3BE03A95F1F70000A59884
:1006200000000000069509F0DDCFA59800E813E072
:100630001023A9F00000A59A0000000000000000AF
:10064000000000000000000000000000A59838E055
:100650003A95F1F700000000069561F0E8CFA59A01
:100660003BE03A95F1F70000A598000000000695E0
:1006700009F0DDCFA59800E8182F1023A9F000009D
:10068000A59A00000000000000000000000000002B
:10069000000000000000A59838E03A95F1F700004E
:1006A0000000069561F0E8CFA59A3BE03A95F1F796
:1006B0000000A59800000000069509F0DDCFA59880
:1006C0000000000000000000A59A000000000000EB
:1006D0000000A59813B31072E9F330E40FE30A9514
:1006E00019F013B31072D9F788278095FF91EF9115
:1006F000C198EF93FF93882700270395B1F09D9948
:10070000FCCFC19808C00027039579F09D99FCCFD4
:10071000839551F001930027039539F09D9BFCCF01
:10072000839511F00193EFCFC19AFF91EF9181383A
:1007300021F081E080938D0012C1DF01AE014757A7
:100740005F4F20E090818181981708F421E02D937C
:100750003296E417F507A9F7FE01319688E0DF012C
:100760001D928A95E9F74981FE01799620E030E0F3
:1007700060E870E08081882339F0CB01022E02C04E
:10078000959587950A94E2F7482B2F5F3F4F319656
:100790002830310579F749834A81FE01B19620E07E
:1007A00030E060E870E08081882339F0CB01022ED0
:1007B00002C0959587950A94E2F7482B2F5F3F4F2B
:1007C00031962830310579F740954A834B81FE01F7
:1007D000B99620E030E060E870E08081882339F04D
:1007E000CB01022E02C0959587950A94E2F7482B1B
:1007F0002F5F3F4F31962830310579F74B834C817D
:10080000FE01F19620E030E060E870E0808188230E
:1008100011F080E007C0CB01022E02C095958795AC
:100820000A94E2F7482B2F5F3F4F3196283031056D
:1008300069F74C834D81FE01F99620E030E060E8D5
:1008400070E08081882339F0CB01022E02C095959B
:1008500087950A94E2F7482B2F5F3F4F3196283057
:10086000310579F740954D834E81FE01EF5BFF4FD7
:1008700020E030E060E870E08081882339F0CB012F
:10088000022E02C0959587950A94E2F7482B2F5FB8
:100890003F4F31962830310579F740954E834F818F
:1008A000FE013C9620E030E061E070E0808188232A
:1008B00039F0CB01022E02C0880F991F0A94E2F78B
:1008C000482B2F5F3F4F31962530310579F7FE01D8
:1008D000729620E030E060E270E08081882339F099
:1008E000CB01022E02C0880F991F0A94E2F7482B11
:1008F0002F5F3F4F31962330310579F74F8348857D
:10090000FE01759620E030E061E070E08081882390
:1009100039F0CB01022E02C0880F991F0A94E2F72A
:10092000482B2F5F3F4F31962430310579F789816D
:1009300080937D008A8180937E008B8180937F00ED
:100940008C81809380008D81809381008E81809343
:1009500082008F81809383004093840080E0C85F91
:10096000DE4F0FB6F894DEBF0FBECDBFCF91DF9143
:100970001F910F91089510928D001FDE90E08091DD
:100980008D00882309F491E0892F08958FB7F8949A
:10099000B99AC198A598AD988FBF0FDE08950F93AF
:1009A0001F93DF93CF93CDB7DEB7C254D0400FB6BD
:1009B000F894DEBF0FBECDBFFE013296982FEF93A5
:1009C000FF9300E8192F1023D1F0000068C0A59A0A
:1009D0000000000000000000000000000000000017
:1009E000000000000000000000000000A5983CE0AE
:1009F0003A95F1F700000000069581F0E3CFA59A43
:100A00003FE03A95F1F70000A598000000000000D3
:100A1000000000000000069509F0D4CFA598000062
:100A20000000000000000000000000000000A59A87
:100A300000000000000000000000000000000000B6
:100A4000000000000000000000000000A59830E257
:100A50000FEF0A9511F113B31072D9F700000000DF
:100A60000000000000000000000000000000000086
:100A70000000000000000000000023B3207221935A
:100A80003A9539F00FEF0A9541F023B3207201F740
:100A9000FACF882704C0832F02C088278095FF9152
:100AA000EF91898389818F3F19F020E030E002C007
:100AB0002FEF3FEFC901CE5BDF4F0FB6F894DEBFDB
:100AC0000FBECDBFCF91DF911F910F9108951FBC35
:100AD00083E08EBD1DBC1CBC109290008DE199E09E
:100AE00090938F0080938E00089508B602FE04C094
:100AF00088B7846088BF1AC08CB59DB526E0853A5A
:100B00009207D0F02AE08C38920718F0875E934065
:100B100002C08DE199E090938F0080938E008091C8
:100B20008E0090918F00845A964030F48DE199E0C8
:100B300090938F0080938E001DBC1CBC88B784608E
:100B400088BF10929000089580919000882369F4E6
:100B50002CB53DB580918E0090918F0028173907F4
:100B600020F081E080939000089580E00895629FD6
:100B7000D001739FF001829FE00DF11D649FE00D95
:100B8000F11D929FF00D839FF00D749FF00D659FF6
:100B9000F00D9927729FB00DE11DF91F639FB00DF5
:100BA000E11DF91FBD01CF011124089597FB092E06
:100BB00005260ED057FD04D014D00AD0001C38F4FE
:100BC00050954095309521953F4F4F4F5F4F089579
:100BD000F6F790958095709561957F4F8F4F9F4F59
:100BE0000895A1E21A2EAA1BBB1BFD010DC0AA1F6E
:100BF000BB1FEE1FFF1FA217B307E407F50720F086
:100C0000A21BB30BE40BF50B661F771F881F991F00
:100C10001A9469F760957095809590959B01AC0149
:100C2000BD01CF010895FB01DC0104C08D9101904D
:100C3000801921F441505040C8F7881B990B089542
:040C4000F894FFCF56
:100C4400FF08000000000000000000C604DD02C927
:080C540002B502BB040100001F
:00000001FF
